:020000040000FA
:10000000FC7F00200D060000FD0500000106000039
:1000100000000000000000000000000000000000E0
:1000200000000000000000000000000005060000C5
:100030000000000000000000090600004D0700005D
:1000400010B5064C2378002B07D1054B002B02D0AE
:10005000044800E000BF0123237010BD5C000020B5
:1000600000000000A818000008B5084B002B03D0C2
:100070000748084900E000BF07480368002B03D089
:10008000064B002B00D0984708BDC046000000007A
:10009000A8180000600000205800002000000000A8
:1000A000154A164B1178002909D115491878097895
:1000B0004118C9B21970802012494003C8611178F3
:1000C0000131C9B211701978F02902D819780929BB
:1000D00009D80B4908784042C0B2087018780978EE
:1000E0004118C9B2197012781B789A4203D1802244
:1000F000044B5203DA6170477800002001000020B1
:10010000000000200044004110B5C3699C07FCD4E6
:1001100003680224A3430360C46901231C42FBD18A
:100120000468234303600368DC07FCD4C46901232B
:100130001C42FBD1C469DC401C42F7D1084B1A4376
:100140000260C3695A07FCD4C0239B0243608181CB
:10015000C3699C07FCD4036802221343036010BDEB
:1001600004000040037EDA07FCD5018570470000DB
:10017000027E01235107FBD5428B1A4207D1428BE5
:10018000DA401A4203D1428B92081A4202D0034B42
:1001900001221A70008DC0B27047C046790000205D
:1001A00070B50368041C988B1A1C0821FF320842A2
:1001B00026D0802099839872112353704021144BCC
:1001C000917150715E68134DC0202E40800506432A
:1001D0005E605E693540284358610F4818600F48DB
:1001E00018615D680E4828408025AD02284358609C
:1001F0005868800B8003586000235171237105E01B
:10020000137ADA0602D5201C00F0DAFA207970BDE4
:1002100098010020FFFFFF8F9800002018010020A8
:10022000FF3F00F0002303714371044B01608360C2
:100230000B78022213430B707047C046A1010000E7
:1002400038B5364B2021DA6901200A43DA61344B94
:1002500006241A7802431A70324B0F221978914300
:1002600019701978214319702F490C7820430870B0
:1002700019780A401A701A7860210A431A702B4BB9
:100280002B4A5A805A7852B2002AFBDB294B0121B3
:100290001A780A431A709A78D107FCD42648026863
:1002A000510B1F221140914200D1052111408C01B8
:1002B0001D8D22492940214319850468A10C0A405B
:1002C0001F2A00D11D221C8D1F210A408C4322436E
:1002D0001A8502680721D20D0A408A4200D1032202
:1002E0000A40188D1103164A02400A431A851978EC
:1002F0007F220A401A701A78042112480A431A70A1
:1003000058621A890C218A431A811A8901218A4369
:100310001A810021802201F046F938BD0004004016
:10032000584400413C44004159440041000C004005
:100330000640000000500041246080003FF8FFFFAD
:10034000FF8FFFFF98010020F7B5141C1F4A5F01C3
:1003500001971D1CD319061C5869271C4000400F2B
:1003600003301033C74006D00F1C80225968120694
:100370000A435A6009E02F1C7B1E9F41144BBF01AA
:10038000FF18381C221C01F005F901990F480835A7
:1003900042181761131C5269A104920B890C920335
:1003A0000A435A6159690B4A0A405A616B01F318B2
:1003B0000222DA715979802252420A435A716B0142
:1003C000F318DB799A07FAD5201CFEBD98010020AE
:1003D00018010020FF3F00F0F8B51A4E051C3378D5
:1003E000141C002B12D1184B184A1A645A6C920B29
:1003F00092035A64586C164A02405A64A2235B0066
:10040000EA5C40200243EA54012333704827FF3757
:10041000EA5D0123134012D00B4B5A6C9204920CEC
:10042000A24202D25C6CA404A40C081C221C074942
:1004300001F0B0F80123EB550023337000E01C1CE1
:10044000201CF8BD7A00002098010020D800002070
:10045000FF3F00F0FF3083792022002900D11022D5
:100460001343837170470000084BFF305A69920BA9
:1004700092035A6102230372827980235B42134301
:100480008371037A9A07FCD57047C0469801002013
:1004900080235B421943C9B28172704770B5A023B3
:1004A00003225B00C254134B134A5C6CC0211440FE
:1004B00089050C4346255C64FF35402444550F4DA7
:1004C00030261D6490256D0046555D6B154029430F
:1004D000922559636D0080214155094D1D63B0255A
:1004E0006D0044555C6F22405A67B2235B00C154D3
:1004F00070BDC04698010020FFFFFF8FD80000208C
:1005000058010020024B5B785BB2002BFADB70478E
:10051000000C0040024BDB68DA06FBD57047C04692
:1005200000080040F8B52A4B1E2259689143022268
:1005300011435960274B28491E1C9982998A0A4306
:100540009A82F3680227234C3B42FAD0234D0123C1
:10055000AB60FFF7D7FF224B6B60FFF7D3FF82231F
:10056000DB016B80FFF7CEFFA38C80229343A38433
:10057000FFF7D0FF1B4BE362FFF7CCFFA38C1A4AB7
:100580001343A384FFF7C6FFA38C1F43A784F3681C
:100590001A06FCD50F4BDB685A06F8D50024FFF786
:1005A000B9FFAC60FFF7AEFF104B6B60FFF7AAFF1F
:1005B0000F4B104AC0215A600F4A0906106A000208
:1005C000000A0143116207229C601A60F8BDC04610
:1005D00000400041000800400C060000000C0040F4
:1005E00001050100B805FF7D040A000000070300B3
:1005F00010E000E0E703000000ED00E00EBEFEE7C3
:100600000DBEFEE705BEFEE702BEFEE70E4A0F483E
:1006100038B5824204D10E4A0E4B93420ED10AE005
:100620000D4C9442F7D00023D1188842F3D9E558F5
:1006300004330D60F8E700F011F804E09342FAD2B9
:10064000002102C3FAE7FEE7000000205C00002062
:10065000A80300205C000020AC18000038B5304B27
:100660001A681C1C013221D02E4A191D1160D9B202
:1006700000291BD12C4A1078012210402B4A0AD1A4
:1006800015682B498D4201D110600FE01160294996
:1006900001390029FCD11160226882F30888FF2209
:1006A0009343254A93601E4B5B681847FFF73AFF58
:1006B00062B600F09DFD00F04FF8204B80225203FF
:1006C0009A601F4B1F4A041C5A601B4AC021106AC3
:1006D00009060002000A0143116200229A60072203
:1006E0001A60A368201C9847174B002801D00122EC
:1006F0001A701A78002A05D0002000F08BFA00F05A
:1007000003FBFCE71B78002BEBD100F0E5FD002894
:10071000E7D0012000F07EFA00F0F6FAFCE7C046D0
:10072000002000001802002038040040FC7F002058
:100730003581730748E8010000ED00E00044004106
:1007400010E000E0E70300007B00002008B5FFF7A1
:10075000A7FC00F0C3FA08BD10B5054B054C23609B
:10076000FFF76EFD201C2168FFF75CFD201C10BD0B
:10077000005000411C02002070B5051CC0B0081CD0
:10078000161C0C1C00F017FF40006A4603230230C1
:100790005370107076080123E218013A11785A005C
:1007A000002906D1281C69460023FFF7CDFD40B083
:1007B00070BDB342F6DA684681520133ECE70000BF
:1007C000F7B5BA4A04681378B949271CFF37051CE6
:1007D000102038720B705378B648B74E0370937878
:1007E0003380D178338809020B4333801179B34BBE
:1007F0001980517918880902084318809079B04906
:100800000880D2790888120202430A8040227A7155
:10081000A84F3A78A64F120238780F1C0243A94815
:100820008446181C624500D1C2E020DC80214900CA
:100830008A4200D16EE109DC812A00D192E0822A4D
:1008400000D195E0802A00D064E18BE081235B0039
:100850009A4200D1CFE000DA58E1C0239B009A42CF
:1008600000D157E1984B9A4200D14FE152E19023D9
:100870001B019A4269D015DCD023DB009A4222D0BA
:1008800088231B019A4269D0A023DB009A4200D042
:1008900040E1201CFFF7E8FD3188286889B2FFF7A6
:1008A000F7FD3BE1894B9A4200D12FE100DC31E1B9
:1008B000874B9A4200D11DE1864B9A4200D029E134
:1008C00033886B7122E133881B0A012B08D10B8816
:1008D00012222868934201D80A8892B27E4911E117
:1008E00033881B0A022B08D10B88432228689342C5
:1008F00001D80A8892B2794904E133881B0A032B94
:1009000000D007E13388DBB2012B17D0002B07D0D2
:10091000022B00D0FEE00A882868D2B2704911E0AC
:10092000042201A86F4900F035FE3B8804222868A4
:10093000934201D83A8892B201A9E3E00A88286874
:100940006949D2B2FFF718FFE8E03388201C2B7109
:10095000FFF78AFD201CFFF7A1FDDFE0291C01C97C
:100960000122CFE0614900230B8028680222CAE0FF
:100970005E4900220A801888502210405C4A10709C
:100980001E880F20304018801888032800D9C1E045
:1009900012781B8808335B01E418A379002A01D080
:1009A0009B0600E0DB06DB0F0B8028680222A9E033
:1009B00019887F2291434E4AC9B2117018880F21BD
:1009C000014019803188002900D0A3E0198800294E
:1009D00000D19FE01988032900D99BE012781B8879
:1009E00008335B01E318002A02D020225A718DE0FF
:1009F000102159718AE002887F239A433C4BD2B27E
:100A00001A7001880F220A4002803288002A00D022
:100A100080E00288002A00D17CE00288032A00D905
:100A200078E01B78002B1FD0038808335B01E318A4
:100A30009B799A066AD50388202208335B01E31864
:100A40001A71038808335B01E318DB795F065DD513
:100A50000388402208335B01E318DA71038802221D
:100A600008335B01E3181EE0038808335B01E318D9
:100A70009B79D9064AD50388102208335B01E31815
:100A80001A71038808335B01E318DB799A063DD5B8
:100A90000388202208335B01E318DA7103880122FE
:100AA00008335B01E3181A7130E0C046980000205B
:100AB0007D000020820000208400002086000020AD
:100AC000800000200203000001030000212000003C
:100AD000A121000021220000FC15000004000020DC
:100AE000EC150000DC150000E01500007E00002081
:100AF0007C0000200B8808222868934201D80A88CD
:100B000092B207490023FFF71FFC07E0201CFFF704
:100B1000ABFC03E0201C0121FFF79CFCF7BDC046A5
:100B20004800002007B5054B0122019001A9186873
:100B3000131CFFF709FC01200EBDC0461C0200205B
:100B400013B5054B6C4607341868211C0122FFF7CA
:100B500043FC207816BDC0461C02002010B5074C8F
:100B6000201CFFF71DFB031C0020834205D02268D8
:100B70004823FF33D05C0123184010BD1C02002025
:100B800010B5054A0C1C031C191C10680123221CFB
:100B9000FFF7DAFB201C10BD1C02002070B5084CCA
:100BA000061C201C0D1CFFF7FBFA0023984205D001
:100BB0002068311C2A1CFFF70FFC031C181C70BD99
:100BC0001C020020F8B50C4C051C201C0E1CFFF765
:100BD000E7FA0023271C341C98420AD0002C07D0C7
:100BE000291C221C3868FFF7F7FB241A2D18F5E79B
:100BF000331C181CF8BDC0461C02002008B5031C9D
:100C0000081C111C9847024B64221A8008BDC0467C
:100C10008C000020012805D1054B064A1A60064BBE
:100C2000187004E0002802D1044A014B1A60704792
:100C30008C02002030160000940000207C1600007A
:100C400030B50A1C1C4985B00978031C00292AD03C
:100C5000042A01D1006804E0022A01D1008800E0E2
:100C60000078520004A98B180B3B9C1AA3420BD0AE
:100C70000F210140092902D83025294300E03731EE
:100C800019700009013BF1E701A930230B707823AB
:100C90004B700A208B1898700D20D870074B0432C7
:100CA0001B68D86803E005490968C868191CFFF784
:100CB000A5FF05B030BDC046880000208C02002092
:100CC00072B6EFF30883044A1360036883F308885D
:100CD000436818477047C04690020020084B1A88A6
:100CE000002A03D01A88013A92B21A80054B1A885A
:100CF000002A03D01A88013A92B21A807047C0467F
:100D00008C0000208A000020F0B591B008A9CC4AE0
:100D10000B1C31CA31C351CA51C360CA60C3C94B2D
:100D2000C9489A687A255203520F92005258C7490F
:100D300002609C68A4B262430C60C54900240A604A
:100D4000C44A1460C44C2570C44CC54D2368281C8B
:100D50001B6940219847002802D0C24B64221A80A8
:100D6000C14B00221860C14B1D60C14BC04DBE4F2E
:100D70001A602A683B689A42E6D2BC4B1B681A7814
:100D8000FF2A00D114E2232A00D0EBE1B94E3378D8
:100D9000002B06D0B14BB8491B680222D868FFF778
:100DA0002DFFAD4B1B78532B3CD13B682A689342F7
:100DB0001ED9AE4801322A609A1AB04B01681B68EE
:100DC00001310160AE4E9A4201D2326000E03360E0
:100DD000A04832680068049000F0DCFB33682968A2
:100DE0005A182A60A14A1668F1181160A54A1370B2
:100DF0002B68013B2B609D4B1A68013A1A60A14B8E
:100E00009E4A1B7811688B420AD222689148C91AFF
:100E1000006892699047002802D0924B64221A80A1
:100E2000C0468DE1522B0AD18A48944A2368006853
:100E300011685B69039098476422934B0DE04F2B38
:100E400005D1844B8D4A1B6812681A7078E1482BD3
:100E500005D1804B894A1B6812681A8070E1572BB4
:100E600005D17C4B854A1B6812681A6068E16F2BBC
:100E700003D1784B0121186807E0682B08D1754B26
:100E80007E481B6802211B880360FFF7D9FE57E1EB
:100E9000772B06D16F4B79481B6804211B680360D0
:100EA000F3E7472B13D1754B1868FFF709FF774B12
:100EB0001B6883F3088862B6754B1B78002B00D142
:100EC0003EE1664B06201B681B68984738E1542BAF
:100ED00004D101233370614B1B6864E04E2B0CD1AD
:100EE0003378002B06D15D4B63491B680222D8681A
:100EF000FFF784FE0023337022E1562B57D123687D
:100F00006449D8680122FFF779FE23686249D868EE
:100F10000322FFF773FE614D2368291CD868012264
:100F2000FFF76CFE23685E49D8680D22FFF766FE66
:100F30002368291CD8680122FFF760FE4B4F4C4DF7
:100F40005849002339602B603A1C281C13685E1C2A
:100F500016601B780593002B03D0036801330360F0
:100F6000F4E73E4E2A683368D868FFF747FE3368D7
:100F70004A49D8680122FFF741FE059929604A498C
:100F800039603A4A1368581C10601B78002B04D053
:100F9000374B1A6801321A60F3E733682A68D86859
:100FA000FFF72CFE3368D86833490222C6E0334A83
:100FB000582B17D1244E264D366813682A68B10085
:100FC00093420AD21F4D5808E861384828801D4DC9
:100FD000287DC607FBD55B18F2E7204B34491B6818
:100FE000D868AAE0592B79D112681A4B3149002AE6
:100FF00002D11B680B606CE0124D086819686B68C1
:10100000104E8025AB4392087360002A61D02A4BB2
:101010000C4D2B800B4E337DDD07FBD500230A4D95
:101020002D680195AD08AB4203D3244D054E3580A4
:1010300046E09342F9D09D00465901334E51EEE708
:101040001016000000400041440200203C02002035
:101050003802002088020020340200208C02002088
:10106000480200208A0000202C02002030020020CC
:10107000400200208800002070160000940200202A
:1010800098020020280200208C00002090020020FE
:10109000940000204C160000751600004E1600004B
:1010A00098160000501600005C16000002A5FFFF15
:1010B000651600009000002044A5FFFF04A5FFFF77
:1010C0003F4E357DEE07FBD59D0049194019D21AD8
:1010D0009BE73C4B3C491B68D8682EE05A2B2FD12C
:1010E0003A4B17681D680026EF19BD4206D02878D4
:1010F000311C00F013F90135061CF6E7314B344979
:101100001B680122D868FFF779FD07230F223240C0
:10111000111C36093031092A00DD07311820C018AA
:101120006A468154013BF1D2236806A9D868082297
:10113000FFF764FD23682749D8680322FFF75EFDA7
:10114000254B7A221A70254B00221A60244B1B78FB
:1011500093422DD01B4B23491B680122D868FFF70F
:101160004DFD25E0111C3039C8B21C4B092804D8AC
:101170001D682A01114319601AE0111C4139052923
:1011800003D81E68373A310106E0111C6139052980
:1011900004D81868573A01010A4308E02C2A03D101
:1011A0000A4A1968116001E00B490A7000221A60AE
:1011B0000D4B1A6801321A600C4B1A680132D5E5E2
:1011C000004000418C0200206916000088020020C7
:1011D0006D1600006F1600003402002094020020FB
:1011E000880000207316000040020020300200201A
:1011F00010B51C4B01201A78022402431A701A4BB6
:101200000F221978914319701978214319701749E1
:101210000C782043087019780A401A701A78202137
:101220000A431A70124B04211A6A0A431A62114BBC
:10123000114A5A805A7852B2002AFBDBC4220F4866
:101240000F499203FEF760FF0E4A002313700E4A07
:1012500013700E4A13700E4A13700E4A13700E4A22
:10126000137010BD4A440041354400414B440041D5
:1012700000040040000C0040144000000008004240
:101280002AF600009C020020230300209D0200207B
:10129000A0020020240300202103002008B5C1B2D1
:1012A0000248FEF75FFF012008BDC046000800426B
:1012B000024B187E4007C00F7047C046000800422E
:1012C00008B5FFF7F5FF0028FBD00248FEF750FFF6
:1012D00008BDC0460008004208B5FFF7E9FF00233B
:1012E000984205D0FFF7ECFF031C233B5A425341C1
:1012F000181C08BD70B5041C0D1C4618B44204D05F
:101300002078FFF7CBFF0134F8E7281C70BD10B53B
:10131000041CFFF7D5FF2070012010BD0B0A5840B8
:10132000034B4000C05A0902484080B27047C04693
:10133000A6160000F7B50024051C0F1C261CBC4295
:1013400020D0FFF7BDFF114BC0B21B780190002BDE
:101350001AD1311CFFF7E2FF0D4B061C1A88002A38
:1013600004D10C4A11782A1C002907D001996A1C63
:101370002970802F02D11988013919800134A4B253
:10138000151CDCE7301C00E00120FEBD210300201D
:101390009E02002022030020F0B53E4E85B00022C0
:1013A00003900C1C32703C4B914201D1012201E0B0
:1013B0003A490C801A707F231C4201D080349C4330
:1013C000FFF77EFF3378C0B2002B07D000253570C1
:1013D000FFF776FF3378C0B2AB4236D1432803D053
:1013E000712853D01528EBD1012300930120FFF77A
:1013F00055FF0098FFF752FF00998025C843C0B2FF
:10140000FFF74CFF039B00270293244A1388002B0D
:101410001DD1214901930978002918D10198FFF7BE
:101420003DFF391C0198FFF779FF013D071C002D96
:10143000EBD1000AC0B2FFF731FFF8B2FFF72EFF81
:10144000FFF73EFF3378002B0AD035701FE002997A
:10145000013B09781380029B019101330293DDE780
:10146000C0B2062807D1009B03990133DBB280315B
:101470000093803C0391002CB8D10420FFF70EFFAD
:10148000FFF71EFF044B01251C7000E00025281CFF
:1014900005B0F0BD21030020220300209E020020A1
:1014A000F0B5384C87B0002301902370994201D1E8
:1014B000012301E0344A1180344A6426137043202A
:1014C000FFF7ECFE324FFFF7F3FE002803D1002FA9
:1014D00003D0013FF7E7002F03D1013E002EEED1EC
:1014E0004DE00125FFF7ECFE2378002B38D1C0B288
:1014F0000290012805D004283DD10620FFF7CEFE3A
:1015000039E005AE0221301CFFF714FF019880215D
:10151000FFF710FF23780390002B18D1FFF7D0FEC0
:101520000702FFF7CDFEBFB223783F18BFB2012BF1
:101530000DD0039B9F4207D13378AB4204D1EB43DC
:101540007278DBB29A4204D01820FFF7A7FE00237E
:1015500003E00620FFF7A2FE029B2278002A02D0B9
:10156000002626700BE0012B05D1019A6B1C8032FE
:10157000DDB20192B6E7054A002313700126301C44
:1015800007B0F0BD210300209E02002022030020AE
:1015900000350C0010B50023934203D0CC5CC4543A
:1015A0000133F9E710BD031C8218934202D0197071
:1015B0000133FAE770470023C25C0133002AFBD1F4
:1015C000581E7047F8B5C046F8BC08BC9E46704728
:1015D000F8B5C046F8BC08BC9E4670470403090431
:1015E00041726475696E6F204C4C430041726475A2
:1015F000696E6F204D4B52313030300012010002C5
:101600000200004041234E000002010200010000E0
:101610000800000010000000200000004000000052
:101620008000000000010000000200000004000033
:101630009D120000C1120000B1120000F51200005E
:101640000F13000099130000A11400007600200081
:1016500041707220313120323031390031333A302B
:10166000393A353100580A0D00590A0D005A002345
:101670000A0D003E00322E3000000000250B000055
:10168000410B00005D0B0000810B00009D0B000072
:10169000810B0000C50B00005B41726475696E6FC1
:1016A0003A58595A5D0000002110422063308440AE
:1016B000A550C660E770088129914AA16BB18CC121
:1016C000ADD1CEE1EFF13112100273325222B55298
:1016D0009442F772D662399318837BB35AA3BDD371
:1016E0009CC3FFF3DEE36224433420040114E66468
:1016F000C774A44485546AA54BB528850995EEE5C1
:10170000CFF5ACC58DD55336722611163006D77677
:10171000F6669556B4465BB77AA719973887DFF710
:10172000FEE79DD7BCC7C448E5588668A77840083F
:10173000611802282338CCC9EDD98EE9AFF9488960
:1017400069990AA92BB9F55AD44AB77A966A711AD7
:10175000500A333A122AFDDBDCCBBFFB9EEB799BB0
:10176000588B3BBB1AABA66C877CE44CC55C222C27
:10177000033C600C411CAEED8FFDECCDCDDD2AAD00
:101780000BBD688D499D977EB66ED55EF44E133EB7
:10179000322E511E700E9FFFBEEFDDDFFCCF1BBF50
:1017A0003AAF599F788F8891A981CAB1EBA10CD12A
:1017B0002DC14EF16FE18010A100C230E320045032
:1017C000254046706760B9839893FBA3DAB33DC3A5
:1017D0001CD37FE35EF3B1029012F322D232354282
:1017E000145277625672EAB5CBA5A89589856EF535
:1017F0004FE52CD50DC5E234C324A01481046674D2
:10180000476424540544DBA7FAB79987B8975FE784
:101810007EF71DC73CD7D326F2369106B016576621
:101820007676154634564CD96DC90EF92FE9C8990C
:10183000E9898AB9ABA94458654806782768C01871
:10184000E1088238A3287DCB5CDB3FEB1EFBF98BE4
:10185000D89BBBAB9ABB754A545A376A167AF10AC1
:10186000D01AB32A923A2EFD0FED6CDD4DCDAABDF4
:101870008BADE89DC98D267C076C645C454CA23C11
:10188000832CE01CC10C1FEF3EFF5DCF7CDF9BAFC4
:10189000BABFD98FF89F176E367E554E745E932E61
:1018A000B23ED10EF01E0000000000000114000046
:1018B0000902430002010080320904000001020213
:1018C0000000052400100104240200052406000184
:1018D0000524010001070583030800FF0904010036
:1018E000020A00000007058102400000070502020D
:1018F0004000000000C20100000008006900000074
:0819000041000000000000009E
:1020000000800020B12400009924000099240000E1
:1020100000000000000000000000000000000000C0
:1020200000000000000000000000000099240000F3
:1020300000000000000000009924000005250000B9
:10204000992400009924000099240000992400009C
:102050009924000099240000992400009D24000088
:10206000992400009924000099240000992400007C
:1020700099240000992400000924000099240000FC
:10208000992400009924000099240000592200009E
:102090000000000099240000992400009924000009
:1020A000992400009924000099240000992400003C
:1020B0000000000010B5064C2378002B07D1054B1B
:1020C000002B02D0044800E000BF0123237010BDA4
:1020D000A000002000000000FC4E0000044B10B5E2
:1020E000002B03D00349044800E000BF10BDC046E8
:1020F00000000000A4000020FC4E000010B50921E3
:10210000014800F079F910BDBC000020044B10B567
:102110001868C0B200F0C6FB024B186010BDC04684
:1021200000000020C000002010B5024800F09EF81A
:1021300010BDC046BC000020F7B50C27404E0193EF
:10214000335C04005BB20D0000924743002B2EDA93
:1021500000230B82EB7BDB09FCD1335D394A013371
:102160005BB23355335D12785BB2DB19934203DA0D
:10217000335D5BB20B2B34DD2F8ABFB2EB7BDB0907
:10218000FCD1314B3149186802F0DEFA304B04378C
:102190005843009B00090C3387424DD280B25B004C
:1021A0005853EB7BDB09FCD1FF33335540E0335C04
:1021B000244A5BB21278DB199342CEDA335C254AAB
:1021C0005BB2DB19DB009B5C5B06C6D5335C002190
:1021D0005BB2DB19DB00985C8006800E00F01CFC13
:1021E000BBE7335D1B4A5BB2DB19DB009B5C5B0624
:1021F00009D5335D01215BB2DB19DB00985C8006F9
:10220000800E00F009FC2A8A92B2EB7BDB09FCD13C
:10221000335D5BB2DF190F4BFF00DF197B68D3180A
:10222000009A9BB20C3252005353EB7BDB09FCD17A
:102230006B461B79AB73F7BDBFB25B005F53B0E772
:10224000C5000020C40000200400002040420F0010
:10225000204E0000C8000020002210B510230249C3
:102260001000FFF769FF10BD0030004270B50C4B45
:1022700005001C780B2C10D8621C1A70094B0470D6
:102280001868094902F060FA084BE4005843084B0B
:1022900000091C196060280070BDFF230370FAE775
:1022A000C40000200400002040420F00DC050000B4
:1022B000C8000020F7B50193037804000E00170052
:1022C0000B2B00D986E0C8B2012100F059FB3F2159
:1022D00032002078404DC3005E5D0A408E431643B5
:1022E0005E558823032296219B00DB1BDF171740D6
:1022F000FF18019B0901C91ACB1713405B189B10EB
:10230000BF10A37067700C2102F01EFA0C23C0B23C
:1023100043431A000C32D900695C490654D4013396
:102320009342F8D100284FD12C4B2D4A5A805A782D
:10233000D209FCD12B4E0232338893433380F37B96
:10234000DB09FCD101333380F37BDB09FCD133881B
:10235000DB07FCD433889BB233804023328813439D
:10236000338080233288DB001343338001233279AA
:1023700013433371F37BDB09FCD11B4B1B491868FA
:1023800002F0E2F90300FA2080005843000980B20D
:102390003083F37BDB09FCD18021154B0903D9671E
:1023A000C023C420134A5B00D150800013581B0285
:1023B0001B0A135010231160737332880E3B1343B2
:1023C0003380F37BDB09FCD140222378DB00E95C1E
:1023D0000A43EA542078FEBDC8000020000C0040EB
:1023E0001C400000003000420400002040420F006A
:1023F00004E100E000E100E09623882210B51B0113
:102400009200FFF757FF10BD10B5024800F075FEAF
:1024100010BDC0462801002013B51249124800F033
:10242000D5FB1249124800F0D1FB1249124800F0C6
:10243000CDFB1249124800F0C9FB1249124800F0C6
:10244000C5FB124C1249200000F0C0FB0123019390
:10245000023300930D220B3321000E4800F0C6FD1D
:1024600013BDC046000800426C030020000C00426F
:1024700074030020001000427C030020001400427E
:1024800084030020001800428C03002094030020E5
:10249000001C004228010020FEE70000034B10B59D
:1024A0001B68002B00D0984710BDC0469C0300203D
:1024B00070B50F490F4CA14204D100F08FF800F025
:1024C000EDFEFEE70C4D00238D42F6D0CA18E81849
:1024D000A24205D3094B8242EFD00949002204E011
:1024E000006804331060F1E704C38B42FCD3E4E7D7
:1024F00000000020A0000020004F0000A0000020ED
:10250000DC09002010B500F066F8002801D100F0C9
:1025100057F810BD014B18607047C0469C0300205F
:10252000014B18687047C046A0030020F7B5134858
:10253000012284461249134C8E68636805689B0E1D
:102540001340019288686268019F920E3A40674684
:102550003F6893420ED1BD420CD186420AD35B192B
:10256000FA254868AD00861B07486B437043000D91
:10257000C018FEBD3D0013000600E3E7A0030020E5
:1025800010E000E000ED00E05555000070B5041EBD
:1025900010D0FFF7CBFF050000F01CF8FFF7C6FFD7
:1025A000054B401B9842F7D9FA23013C9B00ED18DC
:1025B000002CF3D170BDC046E70300007047000057
:1025C00010B5034A13680133136000F0C3FA10BD5D
:1025D000A003002070470020704700001E2270B545
:1025E00046484749436893431C3A134343600823D2
:1025F0008C6923438B61434C434B9C829C8A1443DC
:102600009C82DC681442FCD00124404A1470157886
:10261000254203D055786DB2002DF8DB012494607B
:10262000547864B2002CFBDB394C5460547864B2AB
:10263000002CFBDB8224E4015480547864B2002C2B
:10264000FBDB02249C840E34DD682542FCD0314C37
:10265000DC621024DD682542FCD09D8C2E4C2C437E
:102660009C841024DD682542FCD002249D8C8026A9
:102670002C439C844024DD683542FCD0DD68254233
:10268000F9D01024DD682542FCD0002494605478F1
:1026900064B2002CFBDB214C5460547864B2002CF3
:1026A000FBDB1C6A1E4D2C4080251C621C6AAC435F
:1026B0001C62032393601B4B536053785BB2002B67
:1026C000FBDB0023FF240B72174A4B728B72CB7219
:1026D000164B1A60164B174A1B6811689A065B0165
:1026E000C90E2340520F12020B431343124A1385A3
:1026F000802342681343436070BDC04600400041E0
:10270000000400400C06000000080040000C0040DF
:1027100001050100B905FF7D040A00000007030060
:10272000FFFCFFFF03060100006CDC020400002038
:10273000246080002060800000400042FA21314B7C
:1027400010B51868890001F0FFFF2F4B013898423F
:1027500056D82E492E4A4860C020136A00061B0234
:102760001B0A03431362002407238C600B60802143
:10277000136A09061B021B0A0B431362FC22254B3A
:10278000196A0A431A62FC22196A92010A431A6200
:10279000A022196AD2020A431A62E0B2002101346F
:1027A00000F0EEF8162CF8D11B4B1C005A7852B2F0
:1027B000002AFBDB194A5A80194B1A00597EC909B5
:1027C0000129FBD0E421C90099803F21D970537EB3
:1027D000DB09012BFBD0C02300205B01136190704B
:1027E00000F02EF863785BB2002BFBDB0D4B0E4A3A
:1027F0006380D379DB09012BFBD04123537010BDDB
:10280000FEE7C04604000020FFFFFF0010E000E0EC
:1028100000ED00E000040040000C00401E400000FD
:10282000004000422140000000480042914202D096
:1028300002D98A1AD0407047521A9040FBE7000034
:10284000164A00B51300517EC9090129FBD0013891
:10285000042816D81969124A0A400F211A615A78B9
:102860008A4301F067FF0308060B030011000122F1
:102870000A435A7000BD11000322F9E71100022239
:10288000F6E7F02311691B050B430F211361537801
:102890008B43190002230B435370EBE700400042C7
:1028A000FFFFFFF010B504000E2801D80F34E4B28A
:1028B0000121200000F0DCF81823102163432B4C89
:1028C000E4186156002901D014290DD1284B1800B5
:1028D000DA79D209012AFBD002241A78A2431A70AD
:1028E000C379DB09012BFBD022480300427ED209C9
:1028F000012AFBD01F2402692140A2430A4302613E
:102900005A7ED209012AFBD0022219780A431A7092
:102910005A7ED209012AFBD00222197B0A431A737C
:102920001A7ED207FCD501221A765A7ED209012AD4
:10293000FBD00222197B0A431A731A7ED207FCD5F8
:10294000588B80B25A7ED209012AFBD002211A7814
:102950008A431A705A7ED209012AFBD0064B1A68A4
:10296000064B1968FFF762FF10BDC046B04A000071
:1029700000480042004000420C00002008000020F7
:10298000182330B51D00040045430820204A55197E
:102990002856013014D0032912D808006343D156B9
:1029A000D31801F0C7FE02280E1B5868CB01022184
:1029B000184A9B181A1840321170012282405A603E
:1029C00030BD5868CB010621124A9B181A184032B4
:1029D0001170012282405A609A61F1E75868CB0178
:1029E00006210C4A9B181A184032117001228240AD
:1029F0005A605A61E4E75868CB010221054A9B18E6
:102A00001A1840321170012282409A60D8E7C046FD
:102A1000B04A0000004400411823F0B50824584390
:102A2000114A13181C5701341BD0012635005F686A
:102A30008356BD400D4ADB019A18906805420BD1C0
:102A40000C00601E8441D2194032107834400336A5
:102A5000A400B04320431070044A9B18002901D100
:102A60005D61F0BD9D61FCE7B04A0000004400419B
:102A700018224243F8B52C4E0300B218127A52B213
:102A8000140001320ED0481C00240C280AD801F092
:102A900051FE0720202020202020200B0B0B0B00B4
:102AA000012464422000F8BD092905D10021D8B2D3
:102AB000FFF766FF0024F5E70A2902D1D8B20839EA
:102AC000F6E700240B29EDD1D8B20A39FFF758FFF9
:102AD000E8E718204343F2185568F3562C00134AD0
:102AE000DB016E0817389B18C9B204409E19002CF0
:102AF0000DD00F2430363278090122401143C9B27B
:102B00005B19317040331A7810431870D2E73200E5
:102B10000F27303216785B19BE43314311704033B2
:102B20001A7810431870BDE7B04A00000044004115
:102B300010B50400FFF742FD014B1C6010BDC046FC
:102B4000100000200122024B52421A607047C0461A
:102B500010000020164A10B51368591C26D0013BFE
:102B60001360002B22D172B6124B134A04339342E6
:102B700013D9124A01211000147D0C42FCD02021EF
:102B8000148BFF319B085B0021431183D3610C4BF5
:102B900013800123027D1A42FCD0BFF34F8F094BF3
:102BA000094ADA60BFF34F8FC046FDE710BDC0464B
:102BB000100000200020000003020000004000413F
:102BC00002A5FFFF00ED00E00400FA0500230371F9
:102BD000016070479446F0B59E1E721E9641624693
:102BE000056892072F6836063A4332432A60072564
:102BF00005AC24780068A4012940214342680024E0
:102C0000022B00D05C03114321434160F0BD30B57D
:102C1000C0250368AD031C6812052A402243C02466
:102C20000904A40221401143196003685A6814433F
:102C30005C6030BD0123026811680B4313600368B8
:102C40001A68D207FCD4DA69D207F9D47047022394
:102C5000026811680B4313600268D3699B07FCD4B8
:102C600070470268137E9B0702D40379002BF9D1C9
:102C7000002303717047002203685A83704703687A
:102C8000187E4007C00F70470368187EC009704760
:102C9000802302685B42117E0B4313767047036802
:102CA000588B8007C00F704702230268518B0B437B
:102CB000538370470368187EC007C00F70470368CE
:102CC000188DC0B2704703681A7ED207FCD589B24E
:102CD00019850123037118007047012203689A7552
:102CE0007047012203681A75704700000368214A83
:102CF00030B593422FD0204A93422FD01F4A93429F
:102D00002FD01F4A93422FD01E4A93422FD01E4AE3
:102D100093421FD10E2319220121032599401B48FC
:102D2000C024016099082B40AB40FC359D408900D0
:102D30000918A4000859A843C0259D402B0003434F
:102D40000B518023DB011A43114B5A805A7852B23F
:102D5000002AFBDB30BD09231422DDE70A231522FC
:102D6000DAE70B231622D7E70C231722D4E70D232B
:102D70001822D1E700080042000C00420010004277
:102D80000014004200180042001C004200E100E074
:102D9000000C0040F8B504000F0016001D00FFF7FE
:102DA000A5FF2000FFF746FF1C21BB000B40710769
:102DB0002268090C0B431360842322689375012F4A
:102DC0001AD11021012E00D008390C4B6943186824
:102DD000C00001F0B9FC0722216802408B89520330
:102DE000DB04DB0C13438B81226803049089DB0C2A
:102DF000400B400318439081F8BDC04604000020FA
:102E00000120704710B50368014A1B6A984710BD3E
:102E100013040000FC30006A704787239B00C01831
:102E2000C36880204000C01A70470300FC331A6A50
:102E3000002A03D0DB69C018007D704701204042A2
:102E4000FBE710B504000069FFF7F4FE2200002341
:102E5000FC329361D361136287229200A4186360ED
:102E6000A360E36010BD872310B59B00C218D36830
:102E7000002BFCD10069FFF7F4FE10BD0368002BA6
:102E800002D162B6BFF36F8F7047F0200140303936
:102E9000484248417047F0231B0119408023062017
:102EA0009B0099420AD00133FF330130994205D08B
:102EB000802302385B00994200D0002070470F2029
:102EC00001400020012903D00239481E8141481CDD
:102ED000704700008B23F0B5182685B002919B0047
:102EE0000400C05C330008214343324D1700EB1847
:102EF0005956FFF7BDFD304B0821E05C33004343DA
:102F0000EB185956FFF7B4FD2C4BE25C0393022AF1
:102F100009D11133E05CFF2805D008214643AE19E2
:102F20007156FFF7A5FD8C26B600A05DFF2819D0CD
:102F30000121FFF725FD1822A35D21495A43AB5615
:102F4000AD18DB0158188D21890060501D49012200
:102F50005B188E218900635069688A408F2189003F
:102F600062501A600122029B11002069FFF712FFD4
:102F700039002000FFF78FFF390005002000FFF720
:102F80009EFF390006002000FFF77FFF330000900E
:102F9000290020690122FFF71DFE0B4B2069E25C2E
:102FA000039BE15CFFF733FE2069FFF750FE05B09D
:102FB000F0BDC046B04A00002D0200002F02000004
:102FC00018440041144400412E020000802210B534
:102FD00004005200002101F084FC23000022FC3395
:102FE0005A6020009A60DA6010BD0000F7B51D003D
:102FF00008AB1B780400009309AB1B781600019303
:1030000000234360FA239B008360114B0F000833B9
:1030100003601430FFF7DAFF20002130FF30FFF7A4
:10302000D5FF8B236A469B002761E654094B127833
:10303000E554094B2000E2546A46084B1279E254E9
:103040008C22313BFF3B9200A3541032A354FEBDAF
:10305000104E00002D0200002E0200002F02000082
:10306000F7B5EFF3108300930123019372B6802626
:103070000200FF25019BFC327600013B5C1C0FD057
:10308000D4685F1EB44209D05468015554680134B5
:103090002C405460D4680134D460EEE73B00EDE787
:1030A00068460193FFF7EAFEF7BD13B5EFF310830F
:1030B00000930123019372B6019B5A1E0192002BCB
:1030C00015D00300FC33DA68002A0DD09A68845CBE
:1030D0009A680132D2B29A60DA68013ADA606846D8
:1030E000FFF7CCFE200016BD01246442F7E701245F
:1030F0006846FFF7C3FE6442F4E710B504000069B8
:10310000FFF7CDFD002805D02069FFF7D8FD206925
:10311000FFF7CAFD2069FFF7B2FD00281BD0206928
:10312000FFF7CDFD010020001430FFF799FF8C233D
:103130009B00E35CFF2B0ED02300FC331A6A802334
:103140005B009B1A092B06DC8D238F229B009200CB
:10315000E358A2581A602069FFF7ACFD00280ED092
:1031600087239B00E318DB68002B14D0200021305C
:10317000FF30FFF79AFFC1B22069FFF7A4FD206975
:10318000FFF782FD002805D02069FFF781FD206947
:10319000FFF771FD10BD2069FFF7A3FDEFE7000009
:1031A000F8B5040000690D00FFF784FD87239B003C
:1031B000E618002802D0F368002B34D001278022C3
:1031C000F3685200934223D1EFF310833B4210D1B6
:1031D000174B5B68DB05DB0DF1D0103B5BB2002BBE
:1031E00010DAF13A1340083B9B08124A9B009B18E7
:1031F0001B682069FFF75EFD0028E0D02000FFF784
:103200007CFFDCE79B08C0330B4A9B009B58F0E730
:1032100020002130FF302900FFF722FF2069FFF74F
:103220005CFD0120F8BD29002069FFF74CFDF8E79F
:1032300000ED00E01CED00E000E100E010B504004E
:103240001430FFF732FF8C239B00E35CFF2B0ED082
:103250002300FC331A6A80235B009B1A0A2B06DDCD
:103260008E238F229B009200E358A2581A6010BD53
:10327000F7B506000D000C008B180193019B671B2E
:103280009C4207D0336821781B683000984701348E
:103290000028F3D13800FEBD7047000010B5FFF7DD
:1032A0004DFA01F0DDFAFFF7F7FF0120FFF76EF9A5
:1032B000084C200000F014FF200000F057F9FEF742
:1032C0001DFFFEF723FF044B002BFAD000E000BFE8
:1032D000F7E7C046CC03002000000000704710B59F
:1032E000040001F033F8200010BD0000F0B5822981
:1032F00019D1C3B2294D5A01AA189169284C8001ED
:103300000C40C021890521439161264908334018AA
:103310007021506128685B011A5C8A4311003022D9
:103320000A431A54F0BD0029FCD1C026C1B21B4C7F
:103330004B01E3189A681A4DB6052A4032439A6049
:10334000194A800182185A600A0007272468083247
:103350005201115DB9430F000121394311559F6995
:1033600010493D4040182E439E6158617020115D08
:103370008143080010210143115599680B48A21898
:10338000084080214903014399609968890B8903AA
:103390009960402311790B431371C3E7840800201F
:1033A000FFFFFF8FF8030020B8050020FF3F00F06B
:1033B000EFF3108303600123436072B6704773B567
:1033C000836D0400002B1BD10600A83635786846B3
:1033D000FFF7EEFF019BEDB2013B02D33578EDB272
:1033E000FAE768460193FFF749FD002D01D100205F
:1033F00076BD2300A4331868A0342368C01AF7E709
:103400006846FFF7D5FF22000025019BF432013BFF
:1034100002D31578EDB2FAE768460193FFF72EFD67
:10342000002DE4D02300F0331868EC34E5E7000009
:1034300010B5436D4468DBB25A01A218916809487F
:1034400008330840802149030143916091685B0182
:10345000890B890391602268D318402219790A43A5
:103460001A7110BDFF3F00F0F7B5436D4268DBB243
:10347000190004000831106849014118C979C907C9
:1034800011D55B01D21893689B049B0C0CD12000D2
:10349000FFF7CEFF63681A68636DDBB208335B0128
:1034A000D3187F22DA71F7BDE16D002923D1210005
:1034B000A4310B6023000125AC33E56568465360F9
:1034C000FFF776FF260020002100019BA836013B74
:1034D000F430F5315A1C33D0357002785F1ED2B209
:1034E0000A700A78002A04D120000193FFF7A0FF98
:1034F000E8E73B00EEE72100F0310B600023E365D5
:103500002300603353606846FFF752FF0125260011
:1035100020002100019BF436013BA830F5315A1CF4
:103520000ED0357002785F1ED2B20A700A78002A77
:1035300004D120000193FFF77BFFE8E73B00EEE7B3
:1035400068460193FFF79AFCA4E737B56B46DC1D8C
:1035500000230D00237000F0E3FE210000F06EFE5A
:103560002B681818286020783EBD000000780028DD
:1035700010D00121084B1B681A898A431A8108223E
:10358000198B0A431A830422198B0A431A830022D7
:10359000024B1A607047C046840800207C08002057
:1035A00010B50F4A93699B0B9B039361136802222A
:1035B000FF331A729879823A02439A711A7A920703
:1035C000FCD57F24074A2140937A0800A3431900C1
:1035D000802301439172917A5B420B43937210BD39
:1035E000840800200050004110B50C0000F098FE47
:1035F000210000F056FE002804D1034A93699B0B7A
:103600009B03936110BDC04684080020F8B50D00EF
:10361000832A19D1CBB23B4C5A01A21891693A487E
:10362000AD010840C02189050143916137492068F7
:103630006D187021083355615B011A5C8A431100D3
:1036400040220A431A54F8BD022A55D1304A8B0051
:103650009858002802D003685B699847F82000F06A
:1036600071FE0400274E2B4B466003604022002170
:10367000083001F036F922000023A032A36465650A
:10368000E3642365A365E3655360D3641372136039
:1036900013654C3213725372FF222B0013405901F1
:1036A00071188868184F08330740C02080053843D8
:1036B0008860306807265B01195CAD00B1430E00DD
:1036C0000321314319542300616D606811404901A1
:1036D000411860334B60616D63680A401B6852019A
:1036E0009B180122FF33997A20000A439A72FFF750
:1036F0009FFE074B5C51A6E711002800FFF7F6FD7F
:10370000A1E7C04684080020FFFFFF8FF8030020D8
:10371000D00300204C4E000070B505000124064B7C
:10372000A200D258002A06D0210028000134FFF759
:103730006DFF0A2CF3D170BDA40300200B4BCAB25D
:103740000B488901C9185301C31859619969083296
:10375000890B89039961036852019A180223D37176
:103760005179823B0B4353717047C046F8030020E8
:1037700084080020084B8A00D05810B5002803D0D8
:1037800003689B68984710BDC9B2044B490159189A
:1037900088688004800CF6E7D003002084080020AD
:1037A00010B50C00FFF7E6FF00280CD0064BE4B282
:1037B0001B68083464011C19802362795B4213433F
:1037C00063710223E37110BD84080020F0B51C0072
:1037D0002A4B85B01B6807000D000292002B4AD0CF
:1037E000274B8A00D058002808D0036822005B6865
:1037F000029998470400200005B0F0BD3800FFF79B
:10380000B9FF844204D929003800FFF7B3FF040050
:103810000121EBB21B4E03935B010193F2189368F5
:103820009B0B9B039360019A336802989B18FF33AC
:103830005A7A0A435A72144BA901C918220001F09E
:1038400047F8002CD7D029003800FFF793FF002855
:10385000D1D14021039B326808335B01D31818791A
:10386000014319710121D971019BD318FF339A7A51
:103870000A439A72BFE701246442BCE77C08002037
:10388000D003002084080020B805002013B56B4643
:10389000DC1D22000123FFF799FF012801D12078C8
:1038A00016BD01204042FBE770B5CBB2124A134867
:1038B0005C0189018918021951609168104D083323
:1038C0000D40802149032943402591609168890B6F
:1038D0008903916001685A018A1816793543157178
:1038E00095796D06FCD55B01C918CB79DB07FCD552
:1038F00000198068C0B270BDB8050020840800209F
:10390000FF3F00F070B50D0000211400FFF7CCFF61
:10391000A04200D9200000230349A34203D0CA5C7F
:10392000EA540133F9E770BDB8050020F0B51E0078
:103930003A4B85B01B680F000192002B35D08023D5
:10394000DB019E4231D80025354B8A01D318029302
:10395000002E2CD0334B1B680393FF233B401C00ED
:1039600000930834039B64011C19A379DB0921D05F
:103970002D4B2E49186800F0E7FE2D4B17215843B8
:1039800000F0E2FE2B4BE279920713D4DA5D002AB5
:1039900001D10138F7D20122DA55009B5A01214B9F
:1039A0009B189A69920B92039A6101256D42280037
:1039B00005B0F0BD00221F4B3400DA553F2E09D967
:1039C000009B40245A01174B9B18802299691206CC
:1039D0000A439A6122000199029800F079FF009B46
:1039E000A1045A010F4B890C9B18029A2D195A6198
:1039F0009A69361B920B92030A439A61009B039AC1
:103A000008335B01D3180222DA715979823A0A43EA
:103A10005A71019B1B1901939AE7C0467C0800204C
:103A2000F8030020840800200400002040420F001A
:103A300070110100ED03002070B50D001C000D4B4E
:103A4000AE01F61811003000220000F041FFEDB287
:103A500009496D014D196E61AB69084A2000134098
:103A6000AB61AB69A2049B0B920C9B031343AB614C
:103A700070BDC046F803002084080020FF3F00F01E
:103A8000F7B5104B01901B780F001500002B0CD1DF
:103A90000D4B16001C78002C09D00C4E0C483488B5
:103AA0002018641900F014FF34802800FEBD002E99
:103AB000FBD03A19330000210198FFF7BDFF24180D
:103AC000361AF4E778070020790800207A080020E9
:103AD00079070020F8B50F0016000024012A26D926
:103AE000100000F0E1FE0500380000F0BDFF0323E8
:103AF00002220130400028706B7096420DD939784F
:103B000000290AD0531CDBB20137A9549E4203D0CE
:103B10000232EC54D2B2F0E7320029000548FFF738
:103B2000AFFF441EA041C4B2280000F0C7FE200031
:103B3000F8BDC046CC030020F0B50024012685B0B6
:103B4000184B0F0069461E7005000094FFF7FDFC3E
:103B5000154B01A90B806A3BFF3BCB715A330B72AB
:103B6000009B8C7109334B800E4B4E7108711C7099
:103B70003A00092F0FD00D4F09223E700C4E28003D
:103B800000943480FFF77CFF69462800FFF7DDFCD6
:103B9000328808493C702800FFF772FF012005B009
:103BA000F0BDC04678070020090200007908002017
:103BB0007A0800207907002070B5CE7892B0050011
:103BC0000C00022E0BD18B79C9792C4809021943BC
:103BD000FFF7B2FF411E8841C0B212B070BD00F0C5
:103BE0009FFB210000F03EFB002803D0C117081AFC
:103BF000C00FF2E7012E0ED1E279A37912021A4327
:103C00001F49112A13D8D2B2002A10D02800FFF77A
:103C100037FF0120E1E7032EDFD1A378002B08D185
:103C2000E279A37912021A431649032AEBD90A78DA
:103C3000ECE7022B08D1E279A379120212491A4368
:103C40002800FFF747FFC8E7012B05D1E279A379E8
:103C500012021A430D49F3E7032BBED141220100A2
:103C600001A800F03EFE00F05BFB01A900F00AFB9A
:103C7000E279A37912021A4301A9E1E7CC030020FB
:103C8000884E0000784E0000684E00007C4E000018
:103C9000CBB204495B01C9188B699B0B9B038B61F9
:103CA0007047C0468408002037B5050048780C00EE
:103CB0000B2810D800F03EFD061B0F2B0F4045616E
:103CC000494C5A5D097801AA002906D102231180C6
:103CD0002800FFF7B1FE01203EBD00231380284BD2
:103CE0001B78012B00D1137002230021F0E78A78A2
:103CF0000023012A03D101AA1380224BF0E7204AB6
:103D00001370214A93699B0B9B039361E3E78C78C3
:103D1000012C06D100211B4B01AA1C70117023003D
:103D2000D6E70120002CD7D1154B174A187093699C
:103D30009B0B9B039361CFE789782800FFF730FC4A
:103D4000C9E72800FFF738FFC6E701230F4ACCE791
:103D50000B780020DB06BFD12800FFF7DDFCA2783E
:103D60000A4B0B481A6000F0C3FCCAE70123094A5A
:103D7000BBE78A78074B1A60C3E70020ACE7C04670
:103D8000EC030020F4030020840800207C080020BD
:103D900098090020800800203A4BF7B51E780500EE
:103DA000002E5FD1384C23689A8B12070DD508225C
:103DB00031009A833000FFF799FA10222368FF330D
:103DC000997A0A439A72314B1E6023689A8B520784
:103DD00001D504229A83FF331A7A920603D5202252
:103DE000597A0A435A721A7AD20623D569460800CC
:103DF000274AC0CAC0C0A268920B9203A2604022A8
:103E0000587902435A7160230A7828001A422AD14D
:103E1000FFF74AFF2368FF33002827D080229979D3
:103E200052420A439A711A7A520603D54022597AAD
:103E30000A435A727F2601252368FF331E722F0022
:103E4000236808377F01DB19DB79002B07D0114B82
:103E5000AA00D05800280DD003681B689847013588
:103E6000082DECD1F7BDFFF7BFFBD3E720210A4AAD
:103E70009171D8E72900094800F010FC2368DF1988
:103E8000FE71ECE779080020840800207C080020FF
:103E9000B8050020D0030020FF5000419809002001
:103EA00010B50248FFF778FF10BDC046CC030020D4
:103EB00080235B0003800023436007330372704755
:103EC00083000148C0187047A4030020836C402B76
:103ED00009D03F22036CC154036C013313400364C7
:103EE000836C013383647047F7B505006846FFF7BC
:103EF0005FFA00264022019B013B02D32E6D961BE8
:103F0000FAE768460193FEF7B9FFAB6D6846002BF0
:103F10004FD1FFF74DFA2900019BA831013B5A1CF4
:103F20000CD00C785A1EE4B2002C05D168460193DF
:103F3000FEF7A4FF2000FEBD1300F0E768460193E2
:103F40000024FEF79BFF2A002900A0321368A43149
:103F5000B4420ED0086898420BD92800591CEB18BF
:103F60001160603319780830C9B2FFF7AFFF013430
:103F7000E9E709689942DDD1002313600133AB659D
:103F80006846FFF715FA2F002A000021019BA83789
:103F9000013BF532581CC9D0397010785E1E0028DC
:103FA00005D0117028000193FFF742FAEBE73300C8
:103FB000F0E7FFF7FDF92900019BF431013B5A1CA2
:103FC00006D00C785A1EE4B2002CAFD01300F6E7EE
:103FD000684601930024FEF751FF2A002900EC32C5
:103FE0001368F031B44202D0086898421DD80968BD
:103FF00099429FD1002368461360AB65FFF7D8F95B
:104000002F002A000021019BF437013BF532581C98
:1040100000D18BE7397010785E1E002811D0117026
:1040200028000193FFF704FAEAE72800591CEB186F
:104030001160AC3319780830C9B2FFF747FF01347B
:10404000CBE73300E3E710B50400FFF74DFF206D29
:1040500010BD10B50400FFF747FF236D002B03D000
:10406000E36CE418207A10BD01204042FBE7F7B56D
:1040700017000E000400FFF737FF6846FFF798F9B6
:104080003F2200259446019B013B5A1C19D0BD429A
:1040900015D2226D002A12D00121226D4942002A38
:1040A0000AD06046E26CA218117AE26C013202403A
:1040B000E264226D013A226571550135E7E7013B63
:1040C000E3E768460193FEF7D9FE2800FEBD000035
:1040D000014B024A1A6070478408002000500041DA
:1040E0002023F7B5474A0500D1690F200B43D36160
:1040F000012245490B7813430B70444B19788143D7
:10410000197006211C782143197041490C7822430B
:104110000A701A7802401A70602219780A431A70DD
:104120003C4B3D4A5A805F78FF09FCD13B48FEF783
:10413000F1F901233A4C3B4E2268300011780B43D1
:10414000137080223900520000F0CBFB2268937874
:10415000DB07FCD456621F26334B1B68590B980CA7
:104160009B01314030405B0FB14200D105211F2837
:1041700000D10238072B00D1043B31408901178D53
:1041800001912A4930400F40019939431185118D21
:104190000700B143080038431085118D1803244BE4
:1041A0007F260B4003430C2013850823D1788143DD
:1041B0000B430321D3702268D3788B4301390B431F
:1041C000D370226813783340137004232268167862
:1041D000334313702268C1241389A4008343154814
:1041E000138103591B021B0A0351802303601378B8
:1041F00011481943012311702B70002100F0E8F8D9
:10420000F7BDC04600040040584400413C44004112
:1042100059440041000C004006400000A13E00004F
:104220008408002088080020246080003FF8FFFFF9
:10423000FF8FFFFF00E100E09809002070B50E003D
:1042400000254468002C0BD0236831005B682000F7
:104250009847002802DB2D18E468F3E701256D423A
:10426000280070BD70B50D004468002C08D023688C
:1042700029009B6820009847002802D1E468F4E7F1
:10428000200070BD70B50D004468002C07D0236875
:1042900029002000DB689847E4682D18F5E72C70AA
:1042A00070BD70B50D004468002C08D0236829004B
:1042B0001B6820009847002802D1E468F4E720003A
:1042C00070BDF8B542788B790D00017A9B18040017
:1042D00000208B4222DC6368834219D1656000268E
:1042E00023786A71EA792B719B182370AB79B342FA
:1042F00013D9AB68B7006078DF19FFF7E1FD3B68C1
:10430000013603606378F6B201336370EEE70B00A9
:10431000D9680029FBD1DD60E1E70120F8BD00008C
:1043200070B50126054D064C2B68334203D12000A1
:10433000FFF7BEFD2E60200070BDC046880900203A
:104340008C09002010B500F0AFFA10BD10B500F0D8
:10435000B5FA10BD0020704770B50F26CB1D01398E
:1043600002003240D5B22C0000093034092A00DDA9
:1043700007341C70013B8B42F2D170BD10B50C00AC
:104380000B4B1868FFF7E8FF21000A4B083118684B
:10439000FFF7E2FF2100084B10311868FFF7DCFF40
:1043A0002100064B18311868FFF7D6FF202010BDFA
:1043B0000CA0800040A0800044A0800048A08000A5
:1043C00008B4024B9C46103808BC60477D4300008F
:1043D000704770473F20704713B56B460268D9712C
:1043E0000733546819000122A04716BD70B50A268C
:1043F0000B7892B06E44023305000B703C22002112
:10440000300000F06EFA394801AC0690384824219B
:104410000790062020776846364AA1742281364AE2
:10442000364BA281FD3AFF3A8018C177684623399E
:104430000630C17768460730C17702A8C1770720E8
:10444000F277032608316944C87703A9CE77102193
:104450002B366E443170092621851F3169440E7058
:104460000CA9053E0E7033212380022369440B7092
:1044700006360DA90E7022493536A1863B216E44C1
:10448000307010A86274E27702703D3269446A4469
:104490000B70137040210022E37023716371A373CA
:1044A00041336B44218719705A702B7DC039A3703A
:1044B000A37263770133DBB2A3776A7D0B200D0013
:1044C00068441543C5773120684403703A23501C73
:1044D0006B441870412302320A436B441A70210066
:1044E00042220848FFF7CCFA12B070BD1001042434
:1044F000020605240904000001020000080B000068
:1045000007050000CC03002008B4024B9C4610387D
:1045100008BC6047ED43000070B5027D0B790C00CC
:1045200000259A420BD10B784E78A12B09D1212E70
:1045300005D107221B491C48FFF7A2FA01352800C4
:1045400070BD212BFBD1202E22D107221549164800
:10455000FFF7D8F99622134BD200196891421DD16A
:10456000DB79DB071AD4FA20FEF7E2FA00210E48C5
:10457000FFF78EFB0125232EE1D1E378A2781B0201
:1045800013430A4A002108481360FFF781FBD6E76E
:10459000222EEFD18A78034BDA71DBE7FEF7D2FAED
:1045A000E4E7C04618000020CC03002014000020DF
:1045B00008B4024B9C46103808BC604719450000FF
:1045C00010B508220021024800F08BF910BDC0464A
:1045D0001800002010B5417D006A0131FFF7CAF8CC
:1045E000034B1B6801335A1E9341181810BDC04677
:1045F0002000002010B5417D006A0231FFF7D0F89D
:1046000010BD10B5417D006A0231FFF797F810BD6B
:1046100070B50D00417D0400130002312A00006ACC
:10462000FFF784F9002801D10123636070BD000009
:1046300010B5054C23685A1C04D103685B69984780
:1046400003002060180010BD20000020074A03006E
:10465000106810B5411C03D001235B42136010BDEC
:10466000597D186A0131FFF711F9F8E720000020A1
:1046700010B5FDF755FFF423FF330024984207D906
:10468000044B0A20DC79631E9C41E4B2FDF77EFFF7
:10469000200010BD18000020002070477047000067
:1046A000FA239B0010B583600F4B0022C3820300E6
:1046B000283383610D4B04004260C26118005033FF
:1046C00023610830631D21622060DA778323A362AF
:1046D000813BE36280332363FFF722FE2100103128
:1046E000FFF7EFFD200010BD030200009C4E00000C
:1046F000022110B5094B1A68437D5B01D318FF33C3
:104700009C7A21439972437D0133DBB25B01D3185C
:104710000122FF33997A0A439A7210BD840800205F
:1047200010B502490248FFF7BBFF10BDCC030020C3
:104730009809002002B4714649084900095C490003
:104740008E4402BC7047C046002243088B4274D39B
:1047500003098B425FD3030A8B4244D3030B8B4282
:1047600028D3030C8B420DD3FF22090212BA030C8B
:104770008B4202D31212090265D0030B8B4219D36C
:1047800000E0090AC30B8B4201D3CB03C01A52418C
:10479000830B8B4201D38B03C01A5241430B8B42D4
:1047A00001D34B03C01A5241030B8B4201D30B03BD
:1047B000C01A5241C30A8B4201D3CB02C01A5241E4
:1047C000830A8B4201D38B02C01A5241430A8B42A7
:1047D00001D34B02C01A5241030A8B4201D30B0290
:1047E000C01A5241CDD2C3098B4201D3CB01C01AAA
:1047F000524183098B4201D38B01C01A52414309B4
:104800008B4201D34B01C01A524103098B4201D3A1
:104810000B01C01A5241C3088B4201D3CB00C01A0E
:10482000524183088B4201D38B00C01A5241430886
:104830008B4201D34B00C01A5241411A00D20146AB
:10484000524110467047FFE701B5002000F006F81E
:1048500002BDC0460029F7D076E770477047C046D2
:1048600070B500260C4D0D4C641BA410A64209D156
:10487000002600F011F90A4D0A4C641BA410A64250
:1048800005D170BDB300EB5898470136EEE7B30091
:10489000EB5898470136F2E7880000208800002096
:1048A000880000209C00002010B5034B0100186810
:1048B00000F06AF810BDC0462400002010B5034B7C
:1048C0000100186800F016F810BDC0462400002052
:1048D000002310B59A4200D110BDCC5CC454013302
:1048E000F8E703001218934200D1704719700133A2
:1048F000F9E7000070B50500002910D00C1F2368EF
:10490000002B00DAE418280000F0B5F81D4A1368FF
:10491000002B05D163601460280000F0ADF870BD75
:10492000A34209D9216860188342F3D118685B68F3
:1049300041182160EEE713005A68002A01D0A24214
:10494000F9D919685818A0420BD1206809185818CD
:1049500019608242E0D110685268411819605A60AB
:10496000DAE7A04202D90C232B60D5E72168601852
:10497000824203D1106852684118216062605C6015
:10498000CAE7C046CC090020032370B5CD1C9D4367
:10499000083506000C2D1ED20C25A9421DD830006A
:1049A00000F069F8254A14682100002919D1244C27
:1049B0002368002B03D1300000F044F82060290068
:1049C000300000F03FF8431C2BD10C233000336043
:1049D00000F052F803E0002DDFDA0C2333600020F2
:1049E00070BD0B685B1B19D40B2B03D90B60CC1863
:1049F000256003E04B688C420DD11360300000F05D
:104A00003BF8200007220B30231D9043C31AE7D048
:104A10005A42E250E4E763600C00EFE70C0049689B
:104A2000C3E70323C41C9C43A042E1D0211A3000F9
:104A300000F008F8431CDBD1C7E7C046CC090020D2
:104A4000D0090020002370B5064C05000800236043
:104A500000F014F8431C03D12368002B00D02B6016
:104A600070BDC046D80900200023C25C0133002A73
:104A7000FBD1581E7047704770470000044A136806
:104A8000002B00D1034B1818106018007047C04667
:104A9000D4090020DC090020F8B5C046F8BC08BCE9
:104AA0009E467047F8B5C046F8BC08BC9E467047A5
:104AB0000000000016000000080000001C000000BC
:104AC000FF000004000406000000000017000000C2
:104AD000080000001C000000FF00010401040700A2
:104AE000000000000A000000080000001C00000098
:104AF000120000010001FF00000000000B00000098
:104B0000080000001C000000130001010101FF006B
:104B1000010000000A000000080000001C00000066
:104B2000FF00000500050A00010000000B00000066
:104B3000080000001C000000FF00010501050B003B
:104B40000000000014000000080000002C0000001D
:104B5000FF00020002000400000000001500000039
:104B6000080000002C000000FF0003000300050007
:104B70000000000010000000020000001C00000007
:104B8000FF00000200020000000000001100000011
:104B90000200000004000000FF00FFFFFFFF010013
:104BA0000000000013000000020000001C000000D4
:104BB000FF0001030103FF000000000008000000E7
:104BC000030000001C0000001000000000001000A6
:104BD00000000000090000000300000004000000C5
:104BE0001100FFFFFFFFFF000100000017000000A1
:104BF0000300000004000000FF00FFFFFFFFFF00B4
:104C00000100000016000000030000000400000086
:104C1000FF00FFFFFFFFFF00000000000200000098
:104C200001000000060000000000FFFFFFFFFF0082
:104C3000010000000200000001000000040000006C
:104C40000A00FFFFFFFF0200010000000300000058
:104C500001000000040000000B00FFFFFFFF030045
:104C60000000000004000000010000001C00000023
:104C7000040000000000FF0000000000050000002C
:104C8000010000001C000000050001000100FF0001
:104C90000000000006000000010000000400000009
:104CA0000600FFFFFFFFFF000000000007000000FC
:104CB00001000000040000000700FFFFFFFFFF00ED
:104CC00000000000180000000600000000000000C6
:104CD000FF00FFFFFFFFFF000000000019000000C1
:104CE0000600000000000000FF00FFFFFFFFFF00C4
:104CF0000000000012000000080000000400000096
:104D0000FF00FFFFFFFFFF000000000003000000A6
:104D10000800000004000000FF00FFFFFFFFFF008D
:104D2000000000000C000000030000000000000074
:104D3000FF00FFFFFFFFFF00000000000D0000006C
:104D40000300000000000000FF00FFFFFFFFFF0066
:104D5000000000000E00000008000000000000003D
:104D6000FF00FFFFFFFFFF00000000000F0000003A
:104D70000300000000000000FF00FFFFFFFFFF0036
:104D8000000000001B000000080000000000000000
:104D9000FF00FFFFFFFFFF00000000001C000000FD
:104DA0000800000000000000FF00FFFFFFFFFF0001
:104DB00001000000080000000800000000000000E2
:104DC000FF00FFFFFFFFFF000100000009000000DF
:104DD0000800000000000000FF00FFFFFFFF0900C7
:104DE00000000000000000000800000000000000BB
:104DF000FF00FFFFFFFFFF000000000001000000B8
:104E00000800000000000000FF00FFFFFFFFFF00A0
:104E10000000000000000000A1310000713200001D
:104E20001B2E0000672E0000152E00003D320000F2
:104E30002B2E0000052E0000D52E0000432E000072
:104E4000012E000000000000000000006934000096
:104E50006F4000004740000053400000DD3200007A
:104E6000DF320000BF33000041726475696E6F204D
:104E70004D4B5231303030000403090441726475E7
:104E8000696E6F204C4C430012010002EF0201409A
:104E900041234E80000101020301000000000000D8
:104EA00000000000D943000011460000D543000077
:104EB000F5450000D54500004D4600003146000094
:104EC000D1430000D3430000C145000071460000FB
:104ED00003460000ED430000554300001945000063
:104EE0007D430000F0FFFFFF00000000B14500001F
:104EF0000945000099460000C14300000000000081
:104F00000F00000040420F000A0000000A000000ED
:104F1000FFFFFFFFFFFFFFFF00C2010000000800CE
:104F2000FFFFFFFF2800002000000000000000003D
:104F30000000000000000000000000000000000071
:104F40000000000000000000000000000000000061
:104F50000000000000000000000000000000000051
:104F60000000000000000000000000000000000041
:104F70000000000000000000000000000000000031
:104F80000000000000000000DD20000029210000DA
:104F900019240000D140000021470000B520000086
:00000001FF
